:10000000602864001720031801282220A801083066
:10001000A300232017200318A80AAB1EA801A20CD6
:10002000A30B0928AB1AA2132320220808003A08C0
:100030008400380884178004841300052B1B3806BD
:10004000FF3E080037172B081F39003EA1002A0881
:10005000053E0318A10A371F40283713A0000230BD
:1000600056204028A301A200FF30A207031CA307CB
:10007000031C5B280330A100E43040203428A10198
:10008000F43EA000A109FE30031C4928A007031874
:100090004628A0076400A10F462800002018502819
:1000A0002018522808000310A10CA00CFF3E0318D2
:1000B000532820085B28831303138312640008006D
:1000C00007309F006400851CB0286400851C6928E7
:1000D00065280130A300F43033206400851C7228A9
:1000E000BD017E2905158316051105308312BA005E
:1000F0000130B8005430AA004030AB0001203A3C37
:10010000031D7E2801202A3C031D7E2801203D3C42
:10011000031D7E2801204A3C031D7E2801203D3C12
:10012000031D7E280120313C031D7E280120653CF3
:10013000031D7E280120BC00831601309B00831222
:100140003C0883169A0004309C0055309D00AA306C
:100150009D009C149C0183120511831605118312C6
:10016000831601309B0001309C0001308312322045
:1001700083161A088312BC00851583168511831215
:100180000530BA000130B8005430AA004030AB004E
:100190000120413C031DC8280120643C031DC828E0
:1001A00001202B3C031DC82801202B3C031DC8281F
:1001B0000120543C031DC82801207E3C031DC82893
:1001C0000120213C031DC8280120C100BE0164009C
:1001D0003E084102031C7D290530BA000130B800F9
:1001E0005430AA004030AB000120C00064003E083B
:1001F0003C02031D7B29640080304002031C072958
:100200008030C00286178316861383120B2986134B
:10021000831686138312640040304002031C1729A2
:100220004030C00206178316061383121B290613DB
:10023000831606138312640020304002031C272912
:100240002030C00286168316861283122B2986124E
:10025000831686128312640010304002031C372973
:100260001030C00206168316061283123B290612AE
:10027000831606128312640008304002031C4729CB
:100280000830C00286158316861183124B29861109
:10029000831686118312640004304002031C572920
:1002A0000430C00206158316061183125B2906115D
:1002B000831606118312640002304002031C672972
:1002C0000230C00286148316861083126B298610B2
:1002D000831686108312640001304002031C7629C5
:1002E000C00306148316061083127A29061083169B
:1002F00006108312C028BE0FE728C0286400851CA2
:1003000082297E2964003D080C3C031D8829BD011B
:1003100064003D08003C031DAD290610831606103D
:100320008312861083168610831206118316061117
:100330008312861183168611831206128316061203
:1003400083128612831686128312061383160613EF
:100350008312861383168613831264003D08013CC2
:10036000031DB629061483160610831264003D0887
:10037000023C031DC329061083160610831286143F
:1003800083168610831264003D08033C031DD029A8
:1003900086108316861083120615831606118312A3
:1003A00064003D08043C031DDD2906118316061177
:1003B0008312861583168611831264003D08053C5E
:1003C000031DEA29861183168611831206168316E9
:1003D0000612831264003D08063C031DF72906122D
:1003E0008316061283128616831686128312640001
:1003F0003D08073C031D042A8612831686128312C9
:10040000061783160613831264003D08083C031D7B
:10041000112A061383160613831286178316861372
:10042000831264003D08093C031D362A0614831616
:1004300006108312861483168610831206158316FF
:1004400006118312861583168611831206168316EB
:1004500006128312861683168612831206178316D7
:1004600006138312861783168613831205158316C7
:1004700005118312851583168511640083123D08CA
:100480000A3C031D632A0610831606108312861089
:1004900083168610831206118316061183128611A5
:1004A0008316861183120612831606128312861291
:1004B000831686128312061383160613831286137D
:1004C00083168613831264003D080B3C031D882AA3
:1004D0000614831606108312861083168610831264
:1004E0000615831606118312861183168611831250
:1004F000061683160612831286128316861283123C
:100500000617831606138312861383168613831227
:100510000130BF0064001A303F020318982A0A30E5
:1005200032206400851C962ABD0A7E29BF0F8A2AC4
:100530000511831605118312851183168511640038
:1005400083123D080A3C031DC52A061483160610B3
:1005500083128614831686108312061583160611DD
:1005600083128615831686118312061683160612C9
:1005700083128616831686128312061783160613B5
:100580008312861783168613831264003D080B3C82
:10059000031DEA2A0610831606108312861483169A
:1005A0008610831206118316061183128615831690
:1005B000861183120612831606128312861683167C
:1005C0008612831206138316061383128617831668
:1005D000861383120130BF0064001A303F020318F3
:1005E000FA2A0A3032206400851CF82ABD0A7E29C6
:0A05F000BF0FEC2A7E296300FB2AEE
:02400E00463F2B
:024202000000BA
:00000001FF
